 mouhid

 Timestamp is 4da2a51d (Mon Apr 11 18:52:13 2011)

 Preferred load address is 10000000

 Start         Length     Name                   Class
 0001:00000000 00000004H .CRT$XCA                CODE
 0001:00000004 00000004H .CRT$XCZ                CODE
 0001:00000008 00000004H .CRT$XIA                CODE
 0001:0000000c 00000004H .CRT$XIZ                CODE
 0001:00000010 00000004H .CRT$XPA                CODE
 0001:00000014 00000004H .CRT$XPZ                CODE
 0001:00000018 00000004H .CRT$XTA                CODE
 0001:0000001c 00000004H .CRT$XTZ                CODE
 0001:00000020 00000566H .rdata                  CODE
 0001:00000588 00000023H .rdata$debug            CODE
 0001:000005ac 00002164H .text                   CODE
 0001:00002710 00000004H .xdata                  CODE
 0001:00002714 00000028H .idata$2                CODE
 0001:0000273c 00000014H .idata$3                CODE
 0001:00002750 00000078H .idata$4                CODE
 0001:000027c8 000000aaH .idata$6                CODE
 0001:00002880 0000006eH .edata                  CODE
 0002:00000000 00000078H .idata$5                DATA
 0002:00000078 00000454H .data                   DATA
 0002:000004cc 00000018H .bss                    DATA
 0003:00000000 00000100H .pdata                  DATA

  Address         Publics by Value              Rva+Base       Lib:Object

 0000:00000000       ___safe_se_handler_count   00000000     <absolute>
 0000:00000000       ___safe_se_handler_table   00000000     <absolute>
 0001:00000000       __xc_a                     10001000     corelib0:crt0init.obj
 0001:00000004       __xc_z                     10001004     corelib0:crt0init.obj
 0001:00000008       __xi_a                     10001008     corelib0:crt0init.obj
 0001:0000000c       __xi_z                     1000100c     corelib0:crt0init.obj
 0001:00000010       __xp_a                     10001010     corelib0:crt0init.obj
 0001:00000014       __xp_z                     10001014     corelib0:crt0init.obj
 0001:00000018       __xt_a                     10001018     corelib0:crt0init.obj
 0001:0000001c       __xt_z                     1000101c     corelib0:crt0init.obj
 0001:0000005c       ??_C@_1BK@BJEDGIOP@?$AA?$CF?$AAs?$AA?3?$AA?5?$AAD?$AAe?$AAt?$AAa?$AAc?$AAh?$AA?$AN?$AA?6?$AA?$AA@ 1000105c     mouhid.obj
 0001:00000078       ??_C@_1CG@JHDABJCF@?$AAM?$AAo?$AAu?$AAs?$AAe?$AAD?$AAe?$AAt?$AAa?$AAc?$AAh?$AAe?$AAd?$AAE?$AAv?$AAe?$AAn?$AAt?$AA?$AA@ 10001078     mouhid.obj
 0001:000000a0       ??_C@_1CG@NNBNONKD@?$AAM?$AAo?$AAu?$AAs?$AAe?$AAA?$AAt?$AAt?$AAa?$AAc?$AAh?$AAe?$AAd?$AAE?$AAv?$AAe?$AAn?$AAt?$AA?$AA@ 100010a0     mouhid.obj
 0001:000000c8       ??_C@_1BK@LFPGKGAH@?$AA?$CF?$AAs?$AA?3?$AA?5?$AAA?$AAt?$AAt?$AAa?$AAc?$AAh?$AA?$AN?$AA?6?$AA?$AA@ 100010c8     mouhid.obj
 0001:000000e4       ??_C@_1CA@OKFACCGM@?$AAM?$AAO?$AAU?$AAH?$AAI?$AAD?$AA?5?$AAD?$AAl?$AAl?$AAE?$AAn?$AAt?$AAr?$AAy?$AA?$AA@ 100010e4     mouhid.obj
 0001:00000108       ??_C@_1EG@HEENEOMI@?$AA?$CF?$AAs?$AA?3?$AA?5?$AAF?$AAa?$AAi?$AAl?$AAe?$AAd?$AA?5?$AAc?$AAr?$AAe?$AAa?$AAt?$AAi?$AAn?$AAg?$AA?5?$AAm?$AAo?$AAu?$AAs?$AAe?$AA?5?$AAt?$AAh?$AAr?$AAe?$AAa?$AAd@ 10001108     mouhid.obj
 0001:00000150       ??_C@_1DE@IIKINMKE@?$AA?$CF?$AAs?$AA?3?$AA?5?$AAL?$AAo?$AAc?$AAa?$AAl?$AAA?$AAl?$AAl?$AAo?$AAc?$AA?5?$AAe?$AAr?$AAr?$AAo?$AAr?$AA?3?$AA?$CF?$AAd?$AA?$AN?$AA?6?$AA?$AA@ 10001150     mouhid.obj
 0001:00000188       ??_C@_1FK@FNONLNGN@?$AA?$CF?$AAs?$AA?3?$AA?5?$AAD?$AAE?$AAB?$AAU?$AAG?$AAC?$AAH?$AAK?$AA?5?$AAf?$AAa?$AAi?$AAl?$AAe?$AAd?$AA?5?$AAi?$AAn?$AA?5?$AAf?$AAi?$AAl?$AAe?$AA?5?$AA?$CF?$AAs?$AA?5?$AAa@ 10001188     mouhid.obj
 0001:000001e8       ??_C@_1JE@JOKKFCFP@?$AAc?$AA?3?$AA?2?$AAw?$AAi?$AAn?$AAc?$AAe?$AAr?$AAo?$AAo?$AAt?$AAs?$AA?2?$AAt?$AAo?$AAp?$AAa?$AAz?$AA?2?$AAw?$AAi?$AAn?$AAc?$AAe?$AA7?$AA0?$AA0?$AA?2?$AAp?$AAl?$AAa@ 100011e8     mouhid.obj
 0001:0000027c       ??_C@_1CA@LBENOBMA@?$AAH?$AAI?$AAD?$AAD?$AAe?$AAv?$AAi?$AAc?$AAe?$AAA?$AAt?$AAt?$AAa?$AAc?$AAh?$AA?$AA@ 1000127c     mouhid.obj
 0001:0000029c       ??_C@_1CK@EJMAOEFN@?$AA?$CF?$AAs?$AA?3?$AA?5?$AAE?$AAx?$AAi?$AAt?$AAi?$AAn?$AAg?$AA?5?$AAt?$AAh?$AAr?$AAe?$AAa?$AAd?$AA?$AN?$AA?6?$AA?$AA@ 1000129c     mouhid.obj
 0001:000002c8       ??_C@_1GM@KAMEMAIN@?$AA?$CF?$AAs?$AA?3?$AA?5?$AAG?$AAe?$AAt?$AAI?$AAn?$AAt?$AAe?$AAr?$AAr?$AAu?$AAp?$AAt?$AAR?$AAe?$AAp?$AAo?$AAr?$AAt?$AA?5?$AAr?$AAe?$AAt?$AAu?$AAr?$AAn?$AAe?$AAd?$AA?5@ 100012c8     mouhid.obj
 0001:00000334       ??_C@_1CA@FPPCBODG@?$AAM?$AAo?$AAu?$AAs?$AAe?$AAT?$AAh?$AAr?$AAe?$AAa?$AAd?$AAP?$AAr?$AAo?$AAc?$AA?$AA@ 10001334     mouhid.obj
 0001:00000354       ??_C@_1DG@LDJIBABC@?$AA?$CF?$AAs?$AA?3?$AA?5?$AAU?$AAn?$AAh?$AAa?$AAn?$AAd?$AAl?$AAe?$AAd?$AA?5?$AAm?$AAe?$AAs?$AAs?$AAa?$AAg?$AAe?$AA?5?$AA?$CF?$AAu?$AA?$AN?$AA?6?$AA?$AA@ 10001354     mouhid.obj
 0001:00000390       ??_C@_1FC@MGAKAGG@?$AA?$CF?$AAs?$AA?3?$AA?5?$AAR?$AAe?$AAc?$AAe?$AAi?$AAv?$AAe?$AAd?$AA?5?$AAi?$AAn?$AAv?$AAa?$AAl?$AAi?$AAd?$AA?5?$AAs?$AAt?$AAr?$AAu?$AAc?$AAt?$AAu?$AAr?$AAe?$AA?5?$AAp@ 10001390     mouhid.obj
 0001:000003e4       ??_C@_1CO@LBEHPIKP@?$AAH?$AAI?$AAD?$AAD?$AAe?$AAv?$AAi?$AAc?$AAe?$AAN?$AAo?$AAt?$AAi?$AAf?$AAi?$AAc?$AAa?$AAt?$AAi?$AAo?$AAn?$AAs?$AA?$AA@ 100013e4     mouhid.obj
 0001:00000414       ??_C@_1BA@LEPJIIOK@?$AAU?$AAn?$AAk?$AAn?$AAo?$AAw?$AAn?$AA?$AA@ 10001414     mouhid.obj
 0001:00000424       ??_C@_1CG@NEOOBILK@?$AAA?$AAl?$AAl?$AAo?$AAc?$AAa?$AAt?$AAe?$AAU?$AAs?$AAa?$AAg?$AAe?$AAL?$AAi?$AAs?$AAt?$AAs?$AA?$AA@ 10001424     mouhid.obj
 0001:00000450       ??_C@_1CG@EAKONFHH@?$AAP?$AAr?$AAo?$AAc?$AAe?$AAs?$AAs?$AAM?$AAo?$AAu?$AAs?$AAe?$AAR?$AAe?$AAp?$AAo?$AAr?$AAt?$AA?$AA@ 10001450     mouhid.obj
 0001:00000478       ??_C@_1GK@KPHAPAKG@?$AA?$CF?$AAs?$AA?3?$AA?5?$AAB?$AAa?$AAd?$AA?5?$AAp?$AAh?$AAy?$AAs?$AAi?$AAc?$AAa?$AAl?$AA?5?$AAm?$AAa?$AAx?$AA?1?$AAm?$AAi?$AAn?$AA?5?$AAf?$AAo?$AAr?$AA?5?$AAm?$AAo?$AAu@ 10001478     mouhid.obj
 0001:000004e4       ??_C@_1CA@LFKNIOKP@?$AAG?$AAe?$AAt?$AAA?$AAx?$AAi?$AAs?$AAM?$AAo?$AAv?$AAe?$AAm?$AAe?$AAn?$AAt?$AA?$AA@ 100014e4     mouhid.obj
 0001:00000508       ??_C@_1GI@FFADIIEP@?$AA?$CF?$AAs?$AA?3?$AA?5?$AAH?$AAI?$AAD?$AA?3?$AA?5?$AAd?$AAx?$AA?5?$AA?$CF?$AA4?$AAd?$AA?0?$AA?5?$AAd?$AAy?$AA?5?$AA?$CF?$AA4?$AAd?$AA?0?$AA?5?$AAd?$AAw?$AAD?$AAa?$AAt?$AAa?$AA?5@ 10001508     mouhid.obj
 0001:00000570       ??_C@_1BG@PCLEONCF@?$AAM?$AAo?$AAu?$AAs?$AAe?$AAE?$AAv?$AAe?$AAn?$AAt?$AA?$AA@ 10001570     mouhid.obj
 0001:000005ac       DllEntry                   100015ac f   mouhid.obj
 0001:0000072c       HIDDeviceAttach            1000172c f   mouhid.obj
 0001:00000cd0       HIDDeviceNotifications     10001cd0 f   mouhid.obj
 0001:000018d4       ?FreeHidMouse@@YAXPAU_HID_MOUSE@@@Z 100028d4 f   mouhid.obj
 0001:00001e1c       SetEvent                   10002e1c f i mouhid.obj
 0001:00001e50       GetCurrentThread           10002e50 f i mouhid.obj
 0001:00001e68       HidP_MaxUsageListLength    10002e68 f   hidparse:HIDPARSE.dll
 0001:00001e78       HidP_GetCaps               10002e78 f   hidparse:HIDPARSE.dll
 0001:00001e88       HidP_GetSpecificValueCaps  10002e88 f   hidparse:HIDPARSE.dll
 0001:00001e98       HidP_UsageListDifference   10002e98 f   hidparse:HIDPARSE.dll
 0001:00001ea8       HidP_GetUsages             10002ea8 f   hidparse:HIDPARSE.dll
 0001:00001eb8       HidP_GetScaledUsageValue   10002eb8 f   hidparse:HIDPARSE.dll
 0001:00001ec8       DriverMouseHookInitialize  10002ec8 f   MouHidStd:StandardMouse.obj
 0001:00001eec       DriverMouseHook            10002eec f   MouHidStd:StandardMouse.obj
 0001:00001f10       CloseHandle                10002f10 f   coredll:COREDLL.dll
 0001:00001f20       CreateEventW               10002f20 f   coredll:COREDLL.dll
 0001:00001f30       DisableThreadLibraryCalls  10002f30 f   coredll:COREDLL.dll
 0001:00001f40       NKDbgPrintfW               10002f40 f   coredll:COREDLL.dll
 0001:00001f50       RegisterDbgZones           10002f50 f   coredll:COREDLL.dll
 0001:00001f60       CreateThread               10002f60 f   coredll:COREDLL.dll
 0001:00001f70       GetLastError               10002f70 f   coredll:COREDLL.dll
 0001:00001f80       LocalAlloc                 10002f80 f   coredll:COREDLL.dll
 0001:00001f90       EventModify                10002f90 f   coredll:COREDLL.dll
 0001:00001fa0       LocalFree                  10002fa0 f   coredll:COREDLL.dll
 0001:00001fb0       SetThreadPriority          10002fb0 f   coredll:COREDLL.dll
 0001:00001fc0       WaitForSingleObject        10002fc0 f   coredll:COREDLL.dll
 0001:00001fd0       mouse_event                10002fd0 f   coredll:COREDLL.dll
 0001:00001fe0       LocalSize                  10002fe0 f   coredll:COREDLL.dll
 0001:00001ff0       _DllEntryCRTStartup        10002ff0 f   corelib0:pegdentry.obj
 0001:0000205c       __security_init_cookie     1000305c f   corelib0:seccinit.obj
 0001:000020f4       __GSHandlerCheck           100030f4 f   corelib0:gshandler.obj
 0001:00002138       __GSHandlerCheckCommon     10003138 f   corelib0:gshandler.obj
 0001:000021dc       __security_check_cookie    100031dc f   corelib0:armsecgs.obj
 0001:000021ec       __gsfailure                100031ec     corelib0:armsecgs.obj
 0001:00002230       exit                       10003230 f   corelib0:cexit.obj
 0001:00002354       _exit                      10003354 f   corelib0:cexit.obj
 0001:00002374       _cexit                     10003374 f   corelib0:cexit.obj
 0001:0000238c       _c_exit                    1000338c f   corelib0:cexit.obj
 0001:000023a4       _initterm                  100033a4 f   corelib0:crt0dat.obj
 0001:000023f0       _cinit                     100033f0 f   corelib0:crt0dat.obj
 0001:00002420       __crt_ExitProcess          10003420 f   corelib0:exitproc_proxy.obj
 0001:0000244c       GetCurrentProcess          1000344c f i corelib0:exitproc_proxy.obj
 0001:00002464       _onexit                    10003464 f   corelib0:onexit.obj
 0001:00002640       atexit                     10003640 f   corelib0:onexit.obj
 0001:00002690       memcpy                     10003690 f   corelib1:COREDLL.dll
 0001:000026a0       __security_gen_cookie2     100036a0 f   corelib1:COREDLL.dll
 0001:000026b0       __report_gsfailure         100036b0 f   corelib1:COREDLL.dll
 0001:000026c0       free                       100036c0 f   corelib1:COREDLL.dll
 0001:000026d0       realloc                    100036d0 f   corelib1:COREDLL.dll
 0001:000026e0       malloc                     100036e0 f   corelib1:COREDLL.dll
 0001:000026f0       _msize                     100036f0 f   corelib1:COREDLL.dll
 0001:00002700       TerminateProcess           10003700 f   coredll:COREDLL.dll
 0001:00002714       __IMPORT_DESCRIPTOR_HIDPARSE 10003714     hidparse:HIDPARSE.dll
 0001:00002728       __IMPORT_DESCRIPTOR_COREDLL 10003728     coredll:COREDLL.dll
 0001:0000273c       __NULL_IMPORT_DESCRIPTOR   1000373c     hidparse:HIDPARSE.dll
 0002:00000000       __imp_EventModify          10004000     coredll:COREDLL.dll
 0002:00000004       __imp__msize               10004004     corelib1:COREDLL.dll
 0002:00000008       __imp_malloc               10004008     corelib1:COREDLL.dll
 0002:0000000c       __imp_realloc              1000400c     corelib1:COREDLL.dll
 0002:00000010       __imp_free                 10004010     corelib1:COREDLL.dll
 0002:00000014       __imp___report_gsfailure   10004014     corelib1:COREDLL.dll
 0002:00000018       __imp___security_gen_cookie2 10004018     corelib1:COREDLL.dll
 0002:0000001c       __imp_CloseHandle          1000401c     coredll:COREDLL.dll
 0002:00000020       __imp_CreateEventW         10004020     coredll:COREDLL.dll
 0002:00000024       __imp_DisableThreadLibraryCalls 10004024     coredll:COREDLL.dll
 0002:00000028       __imp_NKDbgPrintfW         10004028     coredll:COREDLL.dll
 0002:0000002c       __imp_RegisterDbgZones     1000402c     coredll:COREDLL.dll
 0002:00000030       __imp_CreateThread         10004030     coredll:COREDLL.dll
 0002:00000034       __imp_GetLastError         10004034     coredll:COREDLL.dll
 0002:00000038       __imp_LocalAlloc           10004038     coredll:COREDLL.dll
 0002:0000003c       __imp_TerminateProcess     1000403c     coredll:COREDLL.dll
 0002:00000040       __imp_LocalFree            10004040     coredll:COREDLL.dll
 0002:00000044       __imp_SetThreadPriority    10004044     coredll:COREDLL.dll
 0002:00000048       __imp_WaitForSingleObject  10004048     coredll:COREDLL.dll
 0002:0000004c       __imp_mouse_event          1000404c     coredll:COREDLL.dll
 0002:00000050       __imp_LocalSize            10004050     coredll:COREDLL.dll
 0002:00000054       __imp_memcpy               10004054     corelib1:COREDLL.dll
 0002:00000058       \177COREDLL_NULL_THUNK_DATA 10004058     coredll:COREDLL.dll
 0002:0000005c       __imp_HidP_GetScaledUsageValue 1000405c     hidparse:HIDPARSE.dll
 0002:00000060       __imp_HidP_GetUsages       10004060     hidparse:HIDPARSE.dll
 0002:00000064       __imp_HidP_UsageListDifference 10004064     hidparse:HIDPARSE.dll
 0002:00000068       __imp_HidP_GetSpecificValueCaps 10004068     hidparse:HIDPARSE.dll
 0002:0000006c       __imp_HidP_GetCaps         1000406c     hidparse:HIDPARSE.dll
 0002:00000070       __imp_HidP_MaxUsageListLength 10004070     hidparse:HIDPARSE.dll
 0002:00000074       \177HIDPARSE_NULL_THUNK_DATA 10004074     hidparse:HIDPARSE.dll
 0002:00000078       dpCurSettings              10004078     mouhid.obj
 0002:000004c4       __security_cookie          100044c4     corelib0:seccinit.obj
 0002:000004c8       __security_cookie_complement 100044c8     corelib0:seccinit.obj
 0002:000004d8       _exitflag                  100044d8     corelib0:cexit.obj
 0002:000004dc       __onexitend                100044dc     <common>
 0002:000004e0       __onexitbegin              100044e0     <common>

 entry point at        0001:00001ff0

 Static symbols

 0001:00000a64       ?MouseThreadProc@@YAKPAX@Z 10001a64 f   mouhid.obj
 0001:00000e84       ?AllocateUsageLists@@YAHPAU_HID_MOUSE@@I@Z 10001e84 f   mouhid.obj
 0001:00001068       ?DetermineWheelUsage@@YAXPAU_HID_MOUSE@@@Z 10002068 f   mouhid.obj
 0001:000011a8       ?SetButtonFlags@@YAXPAKPAGKPBKK@Z 100021a8 f   mouhid.obj
 0001:00001318       ?ProcessMouseReport@@YAXPAU_HID_MOUSE@@PADK@Z 10002318 f   mouhid.obj
 0001:00001648       ?GetAxisMovement@@YAJPAU_HID_MOUSE@@GPADKPAJ@Z 10002648 f   mouhid.obj
 0001:000017dc       ?MouseEvent@@YAXKKKK@Z     100027dc f   mouhid.obj
 0001:000019a4       ?ValidateHidMouse@@YAXPAU_HID_MOUSE@@@Z 100029a4 f   mouhid.obj
 0001:00002250       doexit                     10003250 f   corelib0:cexit.obj
